:100000000C9462000C94BE1A0C94EB1A0C948A00A7
:100010000C948A000C948A000C948A000C948A0038
:100020000C948A000C948A000C948A000C948A0028
:100030000C948A000C948C0B0C948A000C948A000B
:100040000C94181B0C948A000C94941E0C94D71ECC
:100050000C948A000C948A000C948A000C948A00F8
:100060000C94ED080C948A000000000700020100C7
:100070000003040600000000000000000102040864
:100080001020408001020408102001020408102002
:10009000040404040404040402020202020203032E
:1000A00003030303000000002300260029000000D2
:1000B0000000250028002B0000000000240027007D
:1000C0002A004B2011241FBECFEFD8E0DEBFCDBFEA
:1000D00012E0A0E0B1E0EAE0F3E402C005900D9286
:1000E000AA3CB107D9F714E0AAECB2E001C01D9216
:1000F000A43BB107E1F710E0C4ECD0E004C02297C4
:10010000FE010E946021C23CD107C9F70E948720EE
:100110000C9483210C9400008091B603813019F473
:1001200082E08093B6038091B603833019F484E0B3
:100130008093B6030895A8950895CF93DF93FC01AB
:10014000962F9270862F817060FF20C0992331F026
:100150008091480380831092CA0216C0A091CA02FF
:10016000C091E103C770D0E0CA56DD4F8881A8175F
:1001700010F080E03CC081E08A0F8093CA02B0E0BA
:10018000A850BD4F8C91808381E031C09923C1F08C
:1001900090819093CB021092CA02292F207E2036A4
:1001A00051F490914803923020F390819F71909385
:1001B0008A0393E01AC09E3F39F71092480317C094
:1001C0009091CB029F3F01F79091CA02993288F635
:1001D00021E0290F2093CA023081E92FF0E0E75493
:1001E000FC4F3083293281F691E090934803DF91F0
:1001F000CF910895DC01ED91FC910190F081E02D0B
:1002000009950895DC01ED91FC910190F081E02DBC
:10021000099508952091B7033091B803382748E035
:10022000C901880F991F37FF06C09C0151E225279D
:1002300050E1352701C09C01415091F73093B8033C
:100240002093B70308958436910520F4BC0180E023
:1002500090E017C09C018E3B910528F42A55310986
:10026000AAE0B0E00CC0823D910528F4245B31097E
:10027000A4E6B0E004C02D5C3109A8E5B2E00E941C
:100280009420A4E6B0E09B01AC010E94A320089555
:1002900090E08C599F4F0E942301089587E080933E
:1002A000E20380E28093E30381E28093E40310920F
:1002B000E50386E28093E6038093E70384E280937C
:1002C000E80385E28093E903089560E089E00E94F5
:1002D000261C61E088E00E94261C61E087E00E9405
:1002E000261C60E082E00E94261C61E084E00E94FF
:1002F000261C089542E050E06CE870E080E00E9427
:100300009E1A0895E3E0F0E089E080935700E491BD
:10031000E67081E0E63009F080E00895CF93DF9346
:10032000C82F0E948201882381F0DFB781E080938B
:10033000B503F8940E949B0088E180936000C0930D
:100340006000C1110E949B00DFBFDF91CF91089533
:10035000FC0140A5842F877090E0959587950196C4
:10036000242F217030E0820F931F880F880F08958B
:100370008F929F92AF92BF92CF92DF92EF92FF92B5
:10038000CF93FC01C0A5EC2FE770F0E0EA56FD4FDB
:10039000A081B0E0C7FF03C024E130E002C02FE03D
:1003A00030E0FC0197A183E1989FF0011124E65A07
:1003B000FE4F80809180A280B380A20FB31F20E403
:1003C0003FE14DE750E00E94AE20A50194010E945C
:1003D000E6208C2F887149F469017A01E0EDCE0E98
:1003E000E7E0DE1EE11CF11C1BC0C7FF05C060E496
:1003F0007AE88CE29EE004C060E07EEE8AEB9BE04F
:1004000069017A01F8EBCF0EFBE0DF1EE11CF11C65
:10041000A50194010E94E620C20ED31EE41EF51E23
:10042000C701B60169517C4F8F4F9F4F28EE33E0D3
:1004300040E050E00E94E620A8EEB3E00E94A32036
:10044000CF91FF90EF90DF90CF90BF90AF909F90B3
:100450008F900895DB01FA01582F569590E0248182
:10046000237030E0322F22274081240F311D119656
:100470003C932E9344814C70218130E060E4469F90
:10048000200D311D112413963C932E931297448115
:100490004073228130E060E1469F200D311D112420
:1004A00015963C932E9314974481407C238130E031
:1004B00064E0469F200D311D112417963C932E9326
:1004C0001697359618969F5F591748F680FF47C0D4
:1004D000408142954695469543702DE431E0429F18
:1004E000C001439F900D11240C9611969C938E93FE
:1004F000808190E074E0969587957A95E1F7837016
:100500009927829FA001839F500D929F500D112427
:10051000445F5F4F13965C934E931297808190E0F7
:10052000969587959695879583709927829FA001C8
:10053000839F500D929F500D1124445F5F4F15967D
:100540005C934E93149740814370429FC001439F38
:10055000900D11240C9617969C938E9316970895E0
:10056000803223E0920708F1883E23E0920740F4AE
:100570008F519340E4E096958795EA95E1F70895C9
:10058000803D27E0920718F48C5D934008958839E8
:1005900028E0920768F4885C974074E09695879508
:1005A0007A95E1F78D509C4F089580E090E0089592
:1005B0008FEF93E008958C30910540F4A4E0880F0C
:1005C000991FAA95E1F7885D9C4F0895843F23E029
:1005D000920718F484529C4F0895811524E09207E5
:1005E00040F48657934FF4E0880F991FFA95E1F78E
:1005F000089580E998E008959C0136952795257522
:100600003575821B930B9C012373337396958795E5
:100610009695879583739373820F931F9C0154E083
:10062000369527955A95E1F7280F391F2F703F709F
:1006300041E051E0249FC001259F900D349F900D13
:100640001124892F08955F98882319F00000289AB3
:1006500002C00000289800005F9A000008955F9A89
:10066000000083B15F980000869581700895CF9354
:10067000DF93D82F5C9A5F985C98C8E08D2F8078C4
:100680000E942303DD0FC150C9F75F98DF91CF911E
:1006900008958F770E9437030895CF93DF93D82F63
:1006A000C8E08D2F80780E942303DD0FC150C9F769
:1006B0005F98DF91CF910895CF93DF935F98C8E063
:1006C00080E0D82FDD0F0E942F038D0FC150C9F796
:1006D000DF91CF9108950E9449030E945C035C9AC8
:1006E0000895A1E0B0E0E7E7F3E00C9437218068DB
:1006F00069830E9437036981862F0E944D035C9AAB
:100700002196E2E00C945321CF93C091C203C827F5
:10071000E82FF0E0E754FC4F678589E70E947103FA
:100720006C2F8DE30E9471036C2F82E40E94710391
:10073000CF91089586E20E946B030895CF938BE2D8
:100740000E946B03C82F8CE20E946B03282F30E0BD
:1007500066E0369527956A95E1F744E0C49FC001AD
:100760001124822B932BCF910895CF93DF93EC012B
:100770006C818CE10E9471036D818DE10E94710397
:100780006E818EE10E9471036F8180E20E9471038D
:10079000688581E20E947103698582E20E9471038B
:1007A0006A8583E20E9471036B8584E20E94710373
:1007B0006C8585E20E9471036D858AE20E94710357
:1007C0006E858EE60E9471036F858FE60E9471032D
:1007D000688980E70E947103698981E70E9471033B
:1007E0006A8982E70E947103DF91CF910895CF92C9
:1007F000DF92EF92FF92CF93DF936B017C01C114E4
:1008000088E3D8068CE9E8068CE1F80628F5C701EC
:10081000B60120E836E948E950E00E94E620E90107
:10082000689760E879E687E69FEF0E94B6206C0D36
:100830007D1D8E1D9F1DF2E0660F771F881F991F7B
:10084000FA95D1F721E732E040E050E00E94E6203F
:10085000F22EE32E80E421C0C701B60120E03DE284
:1008600041E351E00E94E620E901689760E073ED02
:100870008EEC9EEF0E94B6206C0D7D1D8E1D9F1D7F
:10088000660F771F881F991F21E732E040E050E094
:100890000E94E620F22EE32E80E66C2F6F71680F27
:1008A00085E70E9471036E2D86E70E9471036F2D0C
:1008B00087E70E947103DF91CF91FF90EF90DF9067
:1008C000CF9008958F929F92AF92BF92CF92DF9276
:1008D000EF92FF92CF93DF93D82F83E00E946B03B8
:1008E0008093B40384E00E946B038093B30360E0C1
:1008F00086E00E94710361E087E00E9471036FE768
:1009000089E00E94710365E08AE00E94710362E160
:100910008BE00E94710365E18CE00E9471036DEF32
:100920008DE00E94710360E08EE00E947103DD2380
:1009300019F087E491E008C02091E00333E1239FA0
:10094000C0011124865A9E4F0E94B5036CE880E3D3
:100950000E9471036FE082E30E94710362E483E30B
:100960000E9471038091E10387FF02C064E101C02E
:100970006AE084E30E9471036AE285E30E947103E6
:100980006DE286E30E94710364ED87E30E947103C8
:1009900060E088E30E94710360E089E30E947103D4
:1009A000D11109C0C090C203D090C303E090C4032A
:1009B000F090C50307C0C5E9CC2EC1ECDC2EED2CB0
:1009C000CEEDFC2ECAE38F2C9924AA24BB24682DDB
:1009D0008C2F0E947103682D85E08C0F0E9471039B
:1009E000FE2CED2CDC2CCC24CF5FCE3361F76FEFE7
:1009F00083E40E9471036FEF84E40E9471036FEF40
:100A000085E40E9471036FEF86E40E947103DD2389
:100A100011F066E002C06091C6038DE60E9471038A
:100A200060E089E70E9471036091C7038AE70E9432
:100A3000710360E083E70E94710360E084E70E9435
:100A40007103D11109C06091BE037091BF03809101
:100A5000C0039091C10304C060EC7AEC89E896E38E
:100A60000E94F703DF91CF91FF90EF90DF90CF903E
:100A7000BF90AF909F908F90089561E087E00E94B3
:100A8000710364E28EE70E94710363E088E00E94D4
:100A9000710360E088E00E94710365E087E00E94D6
:100AA000710362E085E00E94710383E00E946B03A2
:100AB0008093B40384E00E946B038093B303089592
:100AC00083E00E946B038093B40384E00E946B0375
:100AD0008093B30361E087E00E9471036AE070E0F5
:100AE00080E090E00E94911B0E943D050000089567
:100AF000CF92DF92FF920F931F93CF93DF931F92BA
:100B0000CDB7DEB7082F162F8EE399830E947103AD
:100B1000F02EC02E9981D92E8C2D8F19811738F483
:100B2000F60161916F018FE70E947103F5CF64E0D8
:100B300085E00E94710383E00E946B038093B403FD
:100B400084E00E946B038093B3030E946E1B60934A
:100B5000AF037093B0038093B1039093B20369E045
:100B600087E00E94710381E08093B6030F90DF91CC
:100B7000CF911F910F91FF90DF90CF9008950F9329
:100B80001F930E9478058091B603813099F40E94EA
:100B90006E1B0091AF031091B0032091B10330910F
:100BA000B203601B710B820B930B603A7648814055
:100BB000910548F38091B603813031F46AEB71E01E
:100BC0008AE094E00E94301D1F910F9108950F93C9
:100BD0001F938091B603823021F41092B60381E016
:100BE00020C08091B6038130D9F40E946E1B009121
:100BF000AF031091B0032091B1033091B203601B99
:100C0000710B820B930B613A76488140910540F05D
:100C100061E087E00E9471031092B60382E001C098
:100C200080E01F910F910895EF92FF920F931F9311
:100C3000CF93DF938B019C01442737FD4095542FC0
:100C400060E271EA87E090E00E940821E9011C1649
:100C50001D0614F0C1E0D0E0D80120E231EA47E0FF
:100C600050E00E94AE209E01442737FD4095542F4E
:100C70000E940821790100E010E00E151F055CF4C8
:100C8000289ACE010E94B71B2898CE010E94B71B5C
:100C90000F5F1F4FF2CFCDB7DEB7E6E00C944F21C8
:100CA000CF93DF932C9A6091F2037091F3038091BC
:100CB000F4039091F5030E94F70360E089E70E9436
:100CC000710361E070E080E090E00E94911B0E945F
:100CD0009A03C82F61E070E080E090E00E94911BD1
:100CE0000E949A03D0E0C80FD11D61E070E080E05F
:100CF00090E00E94911B0E949A03C80FD11D61E0F1
:100D000070E080E090E00E94911B0E949A032C9872
:100D10009E01280F311DC901969587959695879557
:100D2000DF91CF910895CF93C82F2C9A83E00E9432
:100D30006B038093B40384E00E946B038093B3033E
:100D400060E086E00E94710361E087E00E94710329
:100D50006FE789E00E94710365E08AE00E947103F9
:100D600062E18BE00E94710365E18CE00E947103F7
:100D70006DEF8DE00E94710360E08EE00E947103D0
:100D80006CE280E70E94710360E080E30E947103DF
:100D900060E089E70E94710365E08AE70E947103C1
:100DA00062E181E70E94710362E082E70E947103C1
:100DB00060E083E70E94710360E084E70E947103B2
:100DC0006091F2037091F3038091F4039091F50325
:100DD0000E94F70367E08DE60E9471036AE070E00D
:100DE00080E090E00E94911B69E087E00E9471031F
:100DF0006AE070E080E090E00E94911BCC2369F0F3
:100E0000C5E1C15009F459C061E070E088EB91E0A0
:100E10000E9414060E949B00F4CF61E070E088E815
:100E200091E00E9414060E949B0065E08DE60E94FE
:100E300071036AE070E080E090E00E94911B61E045
:100E400070E088EB91E00E9414060E949B0064E031
:100E50008DE60E9471036AE070E080E090E00E94FD
:100E6000911B61E070E08DE591E00E9414060E9404
:100E70009B0062E08DE60E9471036AE070E080E012
:100E800090E00E94911B61E070E08FEA90E00E9488
:100E900014060E949B0060E08DE60E9471036AE0E8
:100EA00070E080E090E00E94911B62E070E085E0DD
:100EB00091E00E9414060E949B0061E087E00E947E
:100EC00071032C98CF910895CF93DF93EC014AE002
:100ED00050E06D2F70E08AE094E00E94F51D6EE214
:100EE0008AE094E00E94141DBE0184E07695679527
:100EF0008A95E1F76F7077274AE050E08AE094E046
:100F00000E94F51D6EE28AE094E00E94141DBE016D
:100F10006F7077274AE050E08AE094E00E94F51D68
:100F2000DF91CF910895D82FC0E0CD1780F42D9A8E
:100F300064E670E080E090E00E94911B2D9864E6EA
:100F400070E080E090E00E94911BCF5FEECF6CE2FA
:100F500071E080E090E00E94911BE6CF0F931F9319
:100F6000CF93DF93EC01062F15E0115051F0CE0125
:100F70000E946D21081741F0602FCE010E9475215B
:100F8000F4CF82E00E949307DF91CF911F910F91E0
:100F90000895A0E0B0E0EFECF7E00C942921482E92
:100FA000562EC0E0D0E0612C712CE12CF12C00E039
:100FB00010E0442079F081E04816A1F092E0491257
:100FC00019C028E4622E712C30E2E32EF12C0BE4E0
:100FD00013E010C0612C712C6BE1E62EF12C02EEB7
:100FE00013E008C04DE1642E712C59E2E52EF12C7E
:100FF00009EB13E043018C0E9D1E1092B803109272
:10100000B7033401A62CA818B12CC30101966C01BA
:10101000AE14BF04A8F4A00EB11E511006C0C30147
:101020000E946D21F501808305C0F5016081C30137
:101030000E94AE07F50180810E940A013601E2CFCD
:10104000C301511018C0C3010E946D21B82EC60102
:101050000E946D212B2D30E0322F2227282B8091EA
:10106000B7039091B8038217930779F4C0E0D0E0FA
:10107000552453949ECF36016091B8030E94AE0769
:101080006091B703C6010E94AE07D395C13093E0CB
:10109000D90708F48ECF852DCDB7DEB7E0E10C94EB
:1010A000452160E081E00E94C907882331F081E09A
:1010B0009091B903983309F080E0089561E081E0F0
:1010C0000E94C907089561E082E00E94C90708955F
:1010D00060E082E00E94C907811108C0EBE4F3E000
:1010E0001192119283E0EB36F807D1F70895A1E051
:1010F000B0E0EDE7F8E00C94372189830E944E01BF
:1011000092E09093F0039FEF9093F1039AE0909315
:10111000FA031092FB031092FC031092F203109258
:10112000F3031092F4031092F5032EE12093F603DB
:101130009093F70328EB3BE03093F9032093F803F7
:101140008981882371F061E080E00E94C907EBE4A7
:10115000F3E01192119283E0EB36F807D1F70E9489
:1011600063082196E2E00C94532160E080E00E9445
:10117000C907811103C081E00E9477080895CF93C9
:10118000C1E0811101C0C0E06C2F82E10E945F1CB0
:101190006C2F83E10E945F1C1092A9031092A80398
:1011A0008091B9008C6F8093B90080E28093B80081
:1011B00085E48093BC00CF91089585ED8093BC00B9
:1011C0008091BC0084FDFCCF0895ECEBF0E0108230
:1011D00085E480831092A80308951F920F920FB6A2
:1011E0000F9211242F933F934F935F936F937F93AD
:1011F0008F939F93AF93BF93EF93FF93CF93DF931F
:101200001F92CDB7DEB78091B900887F803609F490
:10121000C7C0A8F5883209F464C098F4803109F495
:101220005DC038F4882309F4F3C0883009F456C04F
:10123000F1C0883109F455C0803209F0EBC082E07A
:10124000A7C0803409F477C078F4803309F45FC014
:10125000883309F0DFC084E08093A7038091A8035E
:101260008B7F8093A803D0C0803509F452C08835A5
:1012700009F467C0883409F0CDC085E089C0883999
:1012800009F4C0C0A8F4883709F48AC038F4883655
:1012900009F486C0803709F483C0BCC0883809F4DB
:1012A000B1C0803909F47FC0803809F0B3C07BC079
:1012B000803B09F493C038F4803A09F48CC0883A32
:1012C00009F48CC0A7C0803C09F49EC0883C09F496
:1012D0009BC0883B09F09EC080E081C08091AC0338
:1012E00013C08091A9039FEF980F9093A9038823BF
:1012F000D1F1E091AA03F091AB03CF010196909355
:10130000AB038093AA0380818093BB007DC083E000
:101310003FC0E091AA03F091AB03CF0101969093F7
:10132000AB038093AA038091BB0080838091A903C3
:1013300081508093A9038091A903823008F064C092
:1013400061C0E091AA03F091AB03CF0101969093A5
:10135000AB038093AA038091BB0080838091A90393
:1013600081508093A9038091A8038B7F8093A80369
:101370008091A80380FF4CC08091A8038E7F80934A
:10138000A8038091A80382608093A80384EA3DC0EB
:101390008093A7038091A8038B7F8093A80338C014
:1013A0001092A90331C0E091AD03F091AE033097E4
:1013B00049F18091BB0089838091A90391E0980F46
:1013C0009093A903811102C062E001C060E0CE01E8
:1013D0000196099515C00E94DD0816C081E0E091D4
:1013E000AD03F091AE03309769F0882311F063E00C
:1013F00001C061E0CE010196099599819093BB00EF
:10140000811102C085E801C085EC8093BC0002C058
:101410000E94DD080F90DF91CF91FF91EF91BF9176
:10142000AF919F918F917F916F915F914F913F917C
:101430002F910F900FBE0F901F9018958F929F9233
:10144000AF92BF92CF92DF92EF92FF92CF93DF9352
:10145000EC010E946E1B6B017C014E01A12CB12C92
:101460008091A80382FF11C02097D1F30E946E1BC8
:101470006C197D098E099F0986169706A806B9067C
:1014800078F70E94E50881E004C08091A7031092DC
:10149000A703DF91CF91FF90EF90DF90CF90BF90A7
:1014A000AF909F908F900895A2E0B0E0EAE5FAE057
:1014B0000C943321182F7B01022F047022FD05C0EC
:1014C00080910B0190910C0102C080E090E02A8392
:1014D00049830E941E0A2A814981811136C01092D7
:1014E000A7034093A903F092AB03E092AA03110F64
:1014F0001093AC039091A80321FF02C085E001C0C6
:1015000084E0892B8093A8038091A80381FF0BC0FE
:101510008091A8038D7F8093A8038091AC03809372
:10152000BB0085EC01C085EE8093BC00822F8170EA
:1015300020FF0BC0011105C080910B0190910C019F
:1015400002C080E090E00E941E0A2296E6E00C9421
:101550004F21A2E0B0E0EFEAFAE00C943321182F1B
:101560007B01022F047022FD05C080910B01909138
:101570000C0102C080E090E02A8349830E941E0A89
:101580002A814981811138C01092A7034093A90391
:10159000F092AB03E092AA03812F880F81608093C1
:1015A000AC039091A80321FF02C085E001C084E054
:1015B000892B8093A8038091A80381FF0BC08091A1
:1015C000A8038D7F8093A8038091AC038093BB0018
:1015D00085EC01C085EE8093BC00822F817020FFD6
:1015E0000BC0011105C080910B0190910C0102C04C
:1015F00080E090E00E941E0A2296E6E00C944F21C3
:10160000A0E0B0E0E6E0FBE00C9431210E946E1B0C
:101610000091A3031091A4032091A5033091A60388
:101620006B017C01C01AD10AE20AF30A9701860114
:1016300041E1C41647E2D406E104F10408F442C0D3
:101640002091A20331E0320F3093A20320FF02C0A9
:1016500017E001C010E06093A3037093A40380938C
:10166000A5039093A60363E070E08AE094E00E94F3
:10167000020161E070E08AE094E00E94020107E06C
:10168000010F812F90E0EC01CC0FDD1FC35FDE4F17
:1016900068817981672F772763707727880F991F73
:1016A000880F991F682B792B8AE094E00E94FA003A
:1016B0006881798177278AE094E00E94FA001F5FB1
:1016C0001013DFCFCDB7DEB7E8E00C944D2125B184
:1016D00090E0FC01EE0FFF1FE80FF91FEE5EFC4FDC
:1016E0008081282B25B988B19181892B88B98BB14C
:1016F0009281892B8BB9089585B190910F0389232D
:1017000085B988B190911003892388B98BB19091E4
:10171000110389238BB908951F920F920FB60F9270
:1017200011242F933F934F935F936F937F938F93E6
:101730009F93AF93BF93CF93EF93FF93C0916E03AB
:1017400080910601C81708F03EC080910D0390916A
:101750000E039093870080938600EC2FF0E0EE0F4D
:10176000FF1FE35FFE4F808191810E94DB02880FA3
:10177000991F90930E0380930D0380910D03909118
:101780000E032091070130910801281B390B30937B
:101790000801209307018091F8039091F903880FC5
:1017A000991F2817390720F49093080180930701A7
:1017B00080916C03811142C08091F00380FF41C091
:1017C000C830E0F53EC080910D0390910E039093D8
:1017D0008700809386008091070190910801909383
:1017E0000E0380930D0380916C03882319F08FEF13
:1017F0009FEF06C080910D0390910E038855924093
:1018000090938B0080938A0080E49CE99093080178
:101810008093070180918400909185008097D0F398
:101820000E947C0B80916D03811105C0809106019F
:1018300081500E94670B10926E0327C08FEF9FEFBD
:1018400006C080910D0390910E03885592409093AD
:101850008B0080938A00809184009091850080970E
:10186000D0F30E947C0B80916D03811104C08091A4
:101870006E03811106C080916E038F5F80936E03AB
:1018800004C081500E94670BF6CFFF91EF91CF917A
:10189000BF91AF919F918F917F916F915F914F9188
:1018A0003F912F910F900FBE0F901F90189524E03D
:1018B000829FC00111248C30910538F0853F23E0D0
:1018C000920728F084EF93E008958CE090E008956B
:1018D000CF93DF93C091F103C03390F48C2F8073CA
:1018E00039F0803141F480916F038295807F05C08B
:1018F0008091740302C080917503CF70D0E015C051
:10190000CF33E0F4CF70D0E080916F038295807F79
:101910000E94570CDE01AA0FBB1FA35FBE4F11969A
:101920009C938E932196809175030E94570CFE0123
:10193000EE0FFF1FE35FFE4F91838083DF91CF9116
:10194000089580917003909171039F770E94FC022B
:1019500080936F038F3029F48091750386958058AA
:1019600004C099E0899F802D112480937403F8941A
:101970000E94680C78948091E4038132E1F48091B4
:1019800074039FEF980F9E3F78F08091B0008F7D99
:101990008093B00061E080917403811101C060E028
:1019A00083E00E945F1C08958093B4008091B00092
:1019B00080628093B0000895FF920F931F93CF939E
:1019C000DF9303EE13E0C0E0D0E0B3E0FB2E8C2FFA
:1019D000D801ED918D019E2F907F9031F1F4EF7041
:1019E000F0E0EE0FFF1FE35FFE4F208131816F2D8E
:1019F0000E94C620E92FF0E0EE0FFF1FE057FD4FD9
:101A000061E0808191818217930708F060E0FE0118
:101A1000E256FD4F80810E945F1C2196C730D105A0
:101A2000B1F6CDB7DEB7E5E00C9450210F931F93CC
:101A3000CF93DF930BE413E0C0E0D0E02091F103FB
:101A4000822F8F7090E0C817D907E9F00196C81768
:101A5000D90711F42033B8F4F801808191819F7087
:101A6000892B79F0F894F801808191819F700E9410
:101A7000B002FE01EE0FFF1FE35FFE4F91838083F4
:101A800078940E94DC0C21960E5F1F4FC031D10567
:101A9000A9F6DF91CF911F910F910895FF920F93B7
:101AA0001F93CF93DF9389EB93E00E94A80180936B
:101AB00006019091F103292F2F70281304C081E0B3
:101AC000820F8093060190539F3060F4409106018D
:101AD00030E0842F90E001972817390719F44F5F01
:101AE0004093060180910601813118F080E18093D6
:101AF0000601E4E1F3E0DF0112971C92DF01119788
:101B00001C921082339683E0E932F807A1F74FEF79
:101B10003FEFA7EAB2E003EE13E02FEFE80189916F
:101B20008E018031F8F490E0FD0132976081FC0174
:101B3000EE0FFF1FE80FF91FEE5EFC4F8081862B32
:101B40008083CD010197EC0158818181852B8183B0
:101B50009C918281892B8283609550959095292351
:101B6000352346231396D3E00A3E1D07B9F640936A
:101B70000F033093100320931103CEE9D2E003EE5C
:101B800013E0F12CF80181918F01823230F086321E
:101B9000B8F0863211F460E010C0F5E0FF1204C026
:101BA0008091C1008F7E06C086E0F81205C080914A
:101BB000C100877F8093C10061E088810E94261C5C
:101BC000F3942196E7E0FE12DDCF8091E3038032AB
:101BD00031F461E08AE00E945F1C82E201C082E091
:101BE0008093800081E080936D0380936C038091EB
:101BF000E403813211F08732D9F461E083E00E947E
:101C0000261C60E083E00E945F1C8091E403813227
:101C100031F481E08093B0008093B10009C082E08C
:101C20008093B00085E08093B1008EE38093B30091
:101C30008AE1809381008FEF9FEF90938B008093D8
:101C40008A0080ED97E0909387008093860080E47F
:101C50009CE9909308018093070190930E03809371
:101C60000D0310926E0380916F00816080936F006E
:101C70008091F00383FF0DC080914B0390914C0342
:101C80009F70892B31F00E94160D10926C031092F8
:101C90006D03CDB7DEB7E5E00C945021CF93C82F8C
:101CA0008091E5038B3221F46C2F8EE00E945F1C43
:101CB0008091E403873249F48091B000CC2311F085
:101CC000806101C08F7E8093B000CF910895A2E221
:101CD000B0E0EDE6FEE00C9427216B017C010E9450
:101CE000621B4B015C0181E00E94620483E08093EF
:101CF000B6030E94600566EC71E08AE094E00E9401
:101D0000301D7BE1272EE0E53E2EF7E47F2EA6E492
:101D10004A2EB5E55B2EC114D104E104F10469F04B
:101D20000E94621B681979098A099B096C157D0557
:101D30008E059F0510F080E0D5C08091B6038430F9
:101D400051F764ED71E08AE094E00E94301D8FE766
:101D50000E9449030E945C038AA3823601F509EBC5
:101D600013E00E945C03D8018D938D01B3E0023E25
:101D70001B07B9F78091B903883309F0ADC06DED49
:101D800071E08AE094E00E94301D82E48AA361E061
:101D9000CE0182960E94BF052C9A81E0A3C08037B5
:101DA00041F0893611F581E00E94770889E4898342
:101DB00004C03982C12CD12C76019091B503809159
:101DC000F003992311F0806801C08F778093F003AE
:101DD000E2EEF3E0DE011296822D01900D928A95DB
:101DE000E1F76CE1CE01019675C08437E1F4E4E5DA
:101DF000E98383E08A8388E88B8387E08C838DE0A6
:101E00008D838AE1EDE2F1E0DE01169601900D92FC
:101E10008A95E1F76FE1CE0101960E94BF05C12CC2
:101E2000D12C760159C0853789F402EE13E00E9467
:101E30005C03D8018D938D01B3E00D3F1B07B9F70B
:101E400061E080E00E94C9075AA241C08636B9F419
:101E50004982EBE4F3E0AE014D5F5F4F20813181B9
:101E60003296CA010197DC013C93DA012C934E5F54
:101E70005F4FB3E0EB36FB0789F761E2B3CF8736FC
:101E8000C9F40BE413E00E945C03682E0E945C031B
:101E9000262D30E0322F2227280F311DF801219303
:101EA00031938F01F3E00B361F0769F77AA20E9486
:101EB00063080DC0873481F4EBE4F3E011921192D2
:101EC00083E0EB36F807D1F70E9463087AA261E05D
:101ED000CE0182960E94BF0583E08093B6030E94E4
:101EE0003D0519CFA296E2E10C9443211F93CF93B5
:101EF000DF93C82FD62F61E00E94261C61E08C2F53
:101F00000E945F1C61E08D2F0E945F1C8AE090E0C0
:101F10000E94B71B8D2F0E94921C892B71F060E0EC
:101F20008C2F0E945F1C8AE090E00E94B71B8D2FCF
:101F30000E94921C11E0892B09F010E060E08C2FC8
:101F40000E94261C60E08C2F0E945F1C60E08D2F99
:101F50000E945F1C812FDF91CF911F91089580E433
:101F60008093BA001092BD008DE990E09093AE038B
:101F70008093AD031092480315E004E0C2E0FC2E0C
:101F800080914803813039F480E00E946204F0922D
:101F900048032D98F5CFC0914803C33061F42C98C5
:101FA00080918A030E948403C093B6030E943D057A
:101FB00000934803E5CF80914803843009F780916E
:101FC000B6038430E9F68FE70E944903C8EFD2E0F8
:101FD000E091E103E770F0E0EA56FD4F808190E088
:101FE0009E01285F32402817390724F40E945C03C1
:101FF0008993EECF109348032C9AC2CFAAE2B0E0A7
:10200000E4E0F0E10C9436211FEF198389E2E9EB5B
:10201000F3E0DE01129601900D928A95E1F721E03E
:102020004AE2BE016F5F7F4F80E20E94540A811135
:102030000EC021E041E0BE016F5F7F4F80E20E9451
:10204000A90A811104C082E08093480302C0109362
:10205000480380914803823051F00E94621B6093D4
:102060004403709345038093460390934703AA96D5
:10207000E3E00C945221A1E0B0E0E1E4F0E10C9443
:102080003721809148038230D9F480918A03805AA5
:10209000898321E041E0BE016F5F7F4F80E20E94B3
:1020A000540A882369F08FEF809348030E94621BD3
:1020B00060934403709345038093460390934703D2
:1020C0002196E2E00C945321A1E0B0E0EAE6F0E1D1
:1020D0000C943721809148038230D1F421E041E013
:1020E000BE016F5F7F4F80E20E94A90A882371F0D2
:1020F0008FEF809348030E94621B609344037093A8
:102100004503809346039093470302C0898101C031
:102110008FEF2196E2E00C945321A2E2B0E0E3E9D4
:10212000F0E10C9427219E012F5F3F4F80E1D90100
:102130001D928A95E9F768EE71E08AE094E029A3A0
:102140003AA30E94301D0E9460051D8A1E8A1F8AC4
:10215000188E312C212C00E0812C912C540180EC24
:10216000482E8DE9582E88E5682E85E3782E90E577
:10217000C92E93ECD92EE12CF12C84EF91E0A0E054
:10218000B0E08D8F9E8FAF8FB8A380EC97EFAAEB56
:10219000B7E3898F9A8FAB8FBC8F80EC9DE9A8E560
:1021A000B5E3898B9A8BAB8BBC8B8AE094E00E9461
:1021B000FC1D892B09F4E1C08AE094E00E94291EED
:1021C0009C0133272C32310509F442C0ACF4233290
:1021D000310509F0ABC019821A821B821C821D8254
:1021E0001E821F82188619861A861B861C861D86EB
:1021F0001E861F86188A60C02434310529F02335D5
:10220000310509F4B2C092C064E48AE094E00E940F
:10221000141D2AE030E040EC5DE968E575E38AE0F2
:1022200094E00E94901D6CE28AE094E00E94141DEC
:102230002AE030E040EC57EF6AEB77E38AE094E085
:102240000E94901D6CE28AE094E00E94421DADCF96
:102250000F5F043009F0A9CF29813A814B815C815D
:10226000A8EEB3E00E94A320698B7A8B8B8B9C8BAA
:102270002D813E814F8158850E94A320698F7A8FDE
:102280008B8F9C8F29853A854B855C852D8F3E8F62
:102290004F8F58A32D853E854F8558890E94A320D6
:1022A0006B017C0160323EE473078105910530F4D7
:1022B00062E38CE10E94710300E077CF603345E771
:1022C00074078105910510F462E2F3CF60345CE994
:1022D00075078105910510F466E2EBCF80E5C8161D
:1022E00083ECD806E104F10410F462E1E2CF90E659
:1022F000C9169AEED906E104F10410F465E1D9CFCC
:10230000A0E7CA16A1E1DA06A1E0EA06F10410F49A
:1023100061E0CFCFB0EACB16B6E8DB06B1E0EB0662
:10232000F10410F463E0C5CF65E0C3CF10ED180FE2
:102330001A3008F03ACFE1E0F0E0EC0FFD1F24E0A6
:10234000029FE00DF11D11242081318142815381D2
:10235000AAE0B0E00E94A320610F711D811D911DB4
:10236000608371838283938320CF49885A886B88E6
:102370007C88812C912C540118CF81149104A104E4
:10238000B10489F4C301B2010E94F70361E070E077
:1023900080E090E00E94911B1D8A1E8A1F8A188E81
:1023A000312C22242A948D8D9E8DAF8DB8A1881654
:1023B0009906AA06BB06D0F40E949A032D893E898D
:1023C0004F89588D280F311D411D511D2D8B3E8B7E
:1023D0004F8B588F381608F4382E821508F4282EA3
:1023E0003FEF831A930AA30AB30A56C0C301B2018E
:1023F00028EE33E040E050E00E94E620BA01A90157
:102400002AE030E08AE094E00E94DE1D6CE28AE07F
:1024100094E00E94141D4AE050E0632D8AE094E0AD
:102420000E94ED1D6CE28AE094E00E94141D6D890B
:102430007E898F89988DA50194010E94E620BA01BA
:10244000A9012AE030E08AE094E00E94DE1D6CE2FF
:102450008AE094E00E94141D4AE050E0622D8AE078
:1024600094E00E94ED1D6CE28AE094E00E94421D1F
:102470004C0C5D1C6E1C7F1C898D9A8DAB8DBC8DA8
:1024800084159505A605B70520F449885A886B88F8
:102490007C88812C912C540129893A894B895C894B
:1024A000283E33404105510509F07FCEA296E2E176
:1024B0000C944321A1E0B0E0E0E6F2E10C94372176
:1024C00080E00E948E0161E08CE00E94261C61E0A9
:1024D0008DE00E94261C0E94650160E080E00E9461
:1024E000261C61E081E00E94261C40E052EC61E085
:1024F00070E08AE094E00E94441F0E94B5080E94A8
:10250000680865EF71E08AE094E00E94111D88E898
:1025100093E00E9464076CE072E08AE094E00E941D
:10252000111D4AE050E062E070E08AE094E00E9411
:10253000C61D0E947A0178942D9A62E18EE00E9475
:10254000760F882329F02D982C980E948D10FBCFB0
:1025500063E08AE00E94760F811104C00E94510856
:10256000811119C06FE472E08AE094E00E94111DAD
:1025700060E070E0CB010E94670E882349F00E9462
:102580005E0864E172E08AE094E00E94301D2C9ABB
:102590000E944E0D10C00E944E0D8091E6038232C3
:1025A00009F0C6C08091E703833209F0C1C0809171
:1025B000F00381FDC3C08091E603823231F5809142
:1025C000E703833211F581E00E94BF088091F00398
:1025D00082FF08C06FE272E08AE094E00E94301D42
:1025E0000E94AF0F64E170E080E090E00E94911BD8
:1025F00021E041E0BE016F5F7F4F80E20E94A90AA7
:10260000811103C081E0809348036AE372E08AE0AD
:1026100094E00E94111D8FE00E948E0180E00E94D4
:10262000620410928A0380E00E94840380E0883173
:1026300070F08093CC0283E08093B6030E94600523
:1026400080914803882371F00E94FE0F0BC021E0A7
:10265000280FE82FF0E0E754FC4F9785992349F3C2
:10266000822FE5CF8091E903982F9D7F983229F43E
:1026700040E052EC61E070E023C0893251F42EE278
:1026800040EA56E861E070E08AE094E00E94C51FED
:102690001BC08091E1038871803129F440E855E244
:1026A00060E070E00DC04091BA035091BB036091AF
:1026B000BC037091BD034A3051056105710570F38B
:1026C0008AE094E00E94441F8AE094E00E94FC1D8E
:1026D000892B29F08AE094E00E94291EF5CF809191
:1026E000E803843229F08091C1008F7E8093C1007D
:1026F0008091E903853241F08852833028F080913F
:10270000C100877F8093C1001092CE021092CD024B
:1027100010924A030E946E1B609386037093870396
:1027200080938803909389032196E2E00C945321CF
:102730008091F0038B7F8093F00339CF82FD3BCFF4
:1027400064EF71E080E090E00E94670E882309F456
:1027500032CF0E945E0864E172E08AE094E00E9459
:10276000301D0E944E0D2C9A26CFCF93DF938AE026
:1027700094E00E94FC1D892BE9F0C091CD02D0E0CD
:10278000CE0101968F7199272091CE0230E08217F9
:10279000930781F08AE094E00E94291EC153DD4F27
:1027A00088838091CD0290E001968F719927809364
:1027B000CD02DDCFDF91CF910895A0E0B0E0E3EE50
:1027C000F3E10C943121D82FC62F0E946E1B00918B
:1027D000A3031091A4032091A5033091A6036B01DC
:1027E0007C01C01AD10AE20AF30A9701860141E18D
:1027F000C41647E2D406E104F10408F4D1C16093A1
:10280000A3037093A4038093A5039093A6038091E0
:102810000D0190910E01880F991F80938B03892FD2
:10282000877020918C03287F282B20938C03809124
:102830000F0190911001880F991F382F330F330F1C
:10284000330F2770232B20938C03282F2295269556
:10285000277080918D03807C9770990F990F990F45
:10286000822B892B80938D032091110130911201CD
:10287000220F331F922F9295990F990F907C8F738F
:10288000892B80938D03932F9295990F990F907CAC
:10289000822F86958695892B80938E0332FB88271D
:1028A00080F920918F032E7F282B20938F03809116
:1028B000130190911401880F991F382F330F217045
:1028C000232B20938F03382F331F3327331F20915F
:1028D0009003207F892F8770880F232B282B20932C
:1028E00090038091150190911601880F991F382F40
:1028F0003295307F2F70232B20939003382F329501
:102900003F70209191032078892F87708295807F76
:10291000232B282B2093910380911701909118016C
:10292000880F991F2F7720939103292F279522270E
:1029300027958695822B80939203892F86958370A5
:10294000209193032C7F282B2093930380911901CE
:1029500090911A01880F991F382F330F330F23706E
:10296000232B20939303382F329536953695337069
:1029700020919403207E892F8770880F880F232B46
:10298000282B2093940380911B0190911C01880FA8
:10299000991F382F3295330F307E2F71232B2093C0
:1029A00094039295990F907E869586958695892BAE
:1029B0008093950380911D0190911E01880F991FAE
:1029C00080939603892F877020919703287F282B67
:1029D0002093970380911F0190912001880F991FE8
:1029E000382F330F330F330F2770232B2093970388
:1029F000282F22952695277080919803807C9770C8
:102A0000990F990F990F822B892B8093980320910E
:102A1000210130912201220F331F922F9295990F9D
:102A2000990F907C8F73892B80939803932F9295A5
:102A3000990F990F907C822F86958695892B80938C
:102A4000990332FB882780F920919A032E7F282B47
:102A500020939A038091230190912401880F991F5C
:102A6000382F330F2170232B20939A03382F331FD5
:102A70003327331F20919B03207F892F8770880F76
:102A8000232B282B20939B038091250190912601D5
:102A9000880F991F382F3295307F2F70232B20936A
:102AA0009B03382F32953F7020919C032078892F0B
:102AB00087708295807F232B282B20939C03809105
:102AC000270190912801880F991F2F7720939C034D
:102AD000292F2795222727958695822B80939D0362
:102AE0009695937080919E038C7F892B80939E0393
:102AF0002091290130912A01220F331F922F990F23
:102B0000990F8370892B80939E0322952695269595
:102B1000237080919F03807E932F9770990F990F58
:102B2000822B892B80939F0320912B0130912C01C4
:102B3000220F331F922F9295990F907E8F71892BC0
:102B400080939F03832F8295880F807E26952695FC
:102B50002695282B2093A003DD2311F088E001C0E7
:102B600080E0CC2311F094E001C090E0892B8093A9
:102B7000A1036FE070E08AE094E00E940201CBE8DC
:102B8000D3E069918AE094E00E94561E83E0C23A45
:102B9000D807B9F760E070E08AE094E00E94020193
:102BA000CDB7DEB7E8E00C944D21CF93C82F682F46
:102BB0008AE094E00E94561E8C2F0E940A01CF9159
:102BC0000895A0E0B0E0E7EEF5E10C943121C82FC4
:102BD0000E946E1B0091A3031091A4032091A503F2
:102BE0003091A6036B017C01C01AD10AE20AF30AF4
:102BF0009701860141E1C41647E2D406E104F104DD
:102C000008F445C06093A3037093A4038093A503C5
:102C10009093A6031092B8031092B70388EA0E941B
:102C2000D515CC2311F081E801C081E00E94D515B3
:102C300080E10E94D51500E010E0F801EE0FFF1FC3
:102C4000E35FFE4F808191810E94DB02EC01B3E0E3
:102C5000CC0FDD1FBA95E1F78D2F0E94D5158C2F73
:102C60000E94D5150F5F1F4F0031110531F760919C
:102C7000B80370E08AE094E00E94FA006091B70324
:102C80007091B80377278AE094E00E94FA00CDB7EC
:102C9000DEB7E8E00C944D21AAE1B0E0E2E5F6E110
:102CA0000C9429210E949B008CE00E946B038111EF
:102CB0000BC068E872E08AE094E00E94301D80E07A
:102CC0000E9462040E9460050E94B5130E946E1B60
:102CD0000E94641091E0853009F090E01FEF809130
:102CE000B603843009F406C2911104C284C00E9464
:102CF0009E0390937303809372032C9AC092860371
:102D0000D0928703E0928803F092890310924903DE
:102D100010927A0310927B0310927C0310927D0331
:102D20008091700390917103880F991F8160909337
:102D30007103809370032D9880E00E944E0E809165
:102D4000F802982F9E7309F02CC2F8948091E10349
:102D500049EF52E06DE071E087700E942A020E9404
:102D6000680C78949091F8028091420390FF13C20E
:102D7000811124C09BE4E92E93E0F92E00E010E0DD
:102D8000F7018081918194FD0CC0F801EE0FFF1FC7
:102D9000E35FFE4F808191810E94DB02D7018D931A
:102DA0009C930F5F1F4FB2E0EB0EF11C0031110539
:102DB00039F70E94630881E08093420380914A03BF
:102DC000811103C081E080934A0310926B0310923B
:102DD0006D0310926C038091E103887109F009C2C0
:102DE0000E94DC0C83E08093B6030E943D0581E0E5
:102DF000809343032C980E946E1B4B015C010E9440
:102E0000621B6B017C0180914903823008F063C032
:102E100040908603509087036090880370908903E8
:102E20008091820390918303A0918403B0918503E4
:102E300084159505A605B70509F44DC089EB93E007
:102E40000E94B8016C5D754081099109950184016A
:102E500004191509260937096017710782079307B6
:102E6000D0F5409282035092830360928403709263
:102E700085030E949A03282F80937603809177031D
:102E800090917803820F911D90937803809377033C
:102E9000609179036F5F609379036930E0F070E0CF
:102EA0000E94D2207093780360937703809175031A
:102EB000E3E08E9F600D711D1124769567957695E0
:102EC0006795609375030E94A10C1092780310928D
:102ED00077031092790380914A030091CC028823F2
:102EE00051F110914903101708F029C24090860350
:102EF000509087036090880370908903A501940126
:102F000024193509460957092F8B388F498F5A8F55
:102F100089EB93E00E94B80168517C4F8F4F9F4F1F
:102F20002F89388D498D5A8D62177307840795074D
:102F300008F4CCC104C28091860390918703A091CC
:102F40008803B091890375016401C81AD90AEA0A95
:102F5000FB0A89EB93E00E94B8019B01AC01A02F12
:102F6000B0E00E94A3206C157D058E059F0558F4E6
:102F70008092860390928703A0928803B09289037F
:102F800081E08093430380916C03811116C080918E
:102F9000E903883219F40E94000B0FC0893239F41A
:102FA0006091490380916B030E94DD1306C08A3251
:102FB00021F480916B030E94E115809143038823E3
:102FC00009F472C0E0918A03EF5FE0938A03E8316D
:102FD00031F0F0E0E754FC4F8785811102C0109278
:102FE0008A038091F2039091F303A091F403B091CE
:102FF000F503892B8A2B8B2B09F44EC080917A0321
:1030000090917B03A0917C03B0917D03892B8A2B47
:103010008B2B09F441C00E945006082F10E020912C
:10302000090130910A0136952795369527952C5E32
:103030003F4F2017310770F40E94621B68517C4F8C
:103040008F4F9F4F60937A0370937B0380937C0331
:1030500090937D03C801880F991F880F991F409195
:10306000090150910A019A01220F331F240F351FC5
:10307000820F931F969587959695879590930A0151
:10308000809309016091BE037091BF038091C003DA
:103090009091C1030E94F70380918A030E948403E8
:1030A0000E943B1010924303809148038F3F09F028
:1030B00041C20E94621B009144031091450320917C
:1030C000460330914703601B710B820B930B693EE3
:1030D00073408105910508F42DC20E94621B609324
:1030E00044037093450380934603909347030E94E3
:1030F000FE0F20C20E946E1B6B017C018091B60303
:103100008430D1F48FE70E94490308EF12E0E09188
:10311000E103E770F0E0EA56FD4F808190E098010E
:10312000285F3240281739070CF0E1CD0E945C037C
:10313000D8018D938D01EBCFE091E103E770F0E0D2
:10314000EA56FD4F40814F5F21E0BE016F5F7F4F28
:1031500080E20E94A90A882371F0109348030E941C
:10316000621B6093440370934503809346039093DE
:10317000470390E0B4CDE091E103E770F0E0EA5658
:10318000FD4F408150E0BE016E5F7F4F88EF92E0BF
:103190000E946421B3CD882309F410CE109242031B
:1031A0000DCE982F9873983309F008CE9091EF02C6
:1031B000892787FF03CE90589093EF028091E9030F
:1031C000853209F0FBCD10E0212F30E08091F8022C
:1031D000877090E0821793070CF4F0CD1F5FE12F0A
:1031E000F0E0E850FD4F60818AE094E00E94561EB6
:1031F000EBCF8091EF029091F802982796FD5AC08C
:10320000807C90E489278093EF028091CE023091F8
:10321000CD028317D1F0E0EFF2E020E02F5F90E0E5
:10322000DC01A153BD4F4C91419301968F719927B9
:10323000283011F08313F2CF8093CE02295C809165
:10324000EF02282B2093EF0235C080917603809304
:10325000F0028091E603863251F482E10E94BB1CA9
:1032600095958795959587958093F10202C0109268
:10327000F1028091E703863251F483E10E94BB1C86
:1032800095958795959587958093F20202C0109247
:10329000F20280917203909173039093F3028093F2
:1032A000F40280917003909171039F770E94FC0259
:1032B0008093F50269E08FEE92E00E9478050E940B
:1032C000E70581118DCD0E94B513F9CF8091700370
:1032D00090917103880F991F9093710380937003ED
:1032E00081E080934303111110C0C0927E03D092FD
:1032F0007F03E0928003F092810310927A03109290
:103300007B0310927C0310927D031F5F109349038F
:1033100089EB93E00E94B801640D751D861D971D11
:103320006093860370938703809388039093890347
:103330002D9A81E00E944E0E0E94A10C03C010172E
:1033400009F4A7C080914903882309F41CCE809119
:10335000FA038823D9F090916B03911117C0409123
:103360007E0350917F036091800370918103460139
:103370005701841A950AA60AB70A90E00E94230111
:10338000681579058A059B0508F4B5C08091FC0392
:103390008823D9F090916D03911117C040917E035D
:1033A00050917F0360918003709181034601570122
:1033B000841A950AA60AB70A90E00E9423016815AC
:1033C00079058A059B0508F4ADC08091FB0388232D
:1033D000D9F090916C03911117C040917E035091E8
:1033E0007F03609180037091810346015701841A25
:1033F000950AA60AB70A90E00E942301681579058C
:103400008A059B0508F492C08091F2039091F30322
:10341000A091F403B091F503892B8A2B8B2B09F42F
:10342000B2CD80917A0390917B03A0917C03B091FF
:103430007D030097A105B10509F4A5CDC81AD90AE5
:10344000EA0AFB0AF7FC9FCD8091F0038295817018
:103450000E94930680E00E9462040E943D050E9443
:10346000621B6B017C012091F70330E0A8EEB3E012
:103470000E949420C60ED71EE81EF91E6894C0F85C
:10348000C0927A03D0927B03E0927C03F0927D039A
:103490007ACD8091860390918703A0918803B091A3
:1034A000890324013501481A590A6A0A7B0A89EB03
:1034B00093E00E94B8019B01AC01A12FB0E00E94F3
:1034C000A320641575058605970508F03BCF10927B
:1034D00071031092700381E080934303109275038F
:1034E0000E94A10C8092860390928703A092880389
:1034F000B092890327CF81E080936B030E94160D61
:103500008091F6030E9448016C0D7D1D8E1D9F1D4C
:10351000616060937A0370937B0380937C03909344
:103520007D0334CF81E080936D034FCF81E08093A2
:103530006C036ACF6A96E0E10C9445218230E8F48E
:10354000E82FF0E0EE0FFF1FE350FC4F7183608324
:10355000813041F0809169008C7F842B80936900D9
:10356000E89A089580916900440F551F440F551F34
:10357000837F842B80936900E99A08951F920F92AC
:103580000FB60F9211242F933F934F935F936F9336
:103590007F938F939F93AF93BF93EF93FF9380910C
:1035A000FD039091FE03892B29F0E091FD03F0913A
:1035B000FE030995FF91EF91BF91AF919F918F917C
:1035C0007F916F915F914F913F912F910F900FBE1F
:1035D0000F901F9018951F920F920FB60F92112403
:1035E0002F933F934F935F936F937F938F939F930B
:1035F000AF93BF93EF93FF938091FF0390910004EB
:10360000892B29F0E091FF03F09100040995FF91C7
:10361000EF91BF91AF919F918F917F916F915F914A
:103620004F913F912F910F900FBE0F901F901895C3
:103630001F920F920FB60F9211242F933F938F93E7
:103640009F93AF93BF938091020490910304A09144
:103650000404B09105043091010423E0230F2D37B9
:1036600020F40196A11DB11D05C026E8230F029686
:10367000A11DB11D209301048093020490930304C3
:10368000A0930404B093050480910604909107046C
:10369000A0910804B09109040196A11DB11D809369
:1036A000060490930704A0930804B0930904BF9103
:1036B000AF919F918F913F912F910F900FBE0F90DF
:1036C0001F9018952FB7F89460910204709103042D
:1036D00080910404909105042FBF08953FB7F8949A
:1036E0008091060490910704A0910804B091090408
:1036F00026B5A89B05C02F3F19F00196A11DB11D4D
:103700003FBF6627782F892F9A2F620F711D811D69
:10371000911D42E0660F771F881F991F4A95D1F7C8
:103720000895CF92DF92EF92FF92CF93DF936B01D8
:103730007C010E946E1BEB01C114D104E104F10471
:1037400079F00E946E1B6C1B7D0B683E7340A0F3EA
:1037500081E0C81AD108E108F108C851DC4FECCF6C
:10376000DF91CF91FF90EF90DF90CF900895019778
:10377000009739F0880F991F880F991F02970197BA
:10378000F1F70895789484B5826084BD84B5816032
:1037900084BD85B5826085BD85B5816085BDEEE659
:1037A000F0E0808181608083E1E8F0E01082808138
:1037B00082608083808181608083E0E8F0E08081A6
:1037C00081608083E1EBF0E0808184608083E0EBC6
:1037D000F0E0808181608083EAE7F0E080818460AE
:1037E000808380818260808380818160808380810A
:1037F000806880831092C1000895833081F028F49E
:10380000813099F08230A1F008958630A9F0873098
:10381000B9F08430D1F4809180008F7D03C0809115
:1038200080008F7780938000089584B58F7702C0E1
:1038300084B58F7D84BD08958091B0008F7703C0DB
:103840008091B0008F7D8093B0000895CF93DF9377
:1038500090E0FC01E458FF4F2491FC01E057FF4F3A
:103860008491882349F190E0880F991FFC01E85466
:10387000FF4FA591B49182559F4FFC01C591D49102
:103880009FB7611108C0F8948C91209582238C9386
:10389000888182230AC0623051F4F8948C91322FCF
:1038A000309583238C938881822B888304C0F8947D
:1038B0008C91822B8C939FBFDF91CF910895A1E0D3
:1038C000B0E0E5E6FCE10C943521282F30E0F90169
:1038D000E859FF4F8491F901E458FF4F1491F90121
:1038E000E057FF4F04910023C9F0882321F069833A
:1038F0000E94FD1B6981E02FF0E0EE0FFF1FE255F3
:10390000FF4FA591B4919FB7F8948C91611103C0BA
:103910001095812301C0812B8C939FBF2196E4E0F9
:103920000C945121CF93DF93282F30E0F901E8590F
:10393000FF4F8491F901E458FF4FD491F901E0570A
:10394000FF4FC491CC2391F081110E94FD1BEC2FFD
:10395000F0E0EE0FFF1FEC55FF4FA591B4912C91B5
:103960002D2381E090E021F480E002C080E090E02F
:10397000DF91CF9108958E3008F08E50877020919E
:10398000B90190E4299F90011124822B80937C003F
:1039900080917A00806480937A0080917A0086FD1D
:1039A000FCCF809178002091790090E0922B0895CF
:1039B000A0E0B0E0EEEDFCE10C9431216C017A0165
:1039C000EB01E60EF71E00E010E0CE15DF0561F01A
:1039D0006991D601ED91FC910190F081E02DC60135
:1039E0000995080F191FF1CFC801CDB7DEB7E8E080
:1039F0000C944D216115710589F0DB010D900020BB
:103A0000E9F7AD0141505109461B570BDC01ED911F
:103A1000FC910280F381E02D0995089580E090E00B
:103A200008950E94FA1C0895DC01ED91FC9101902B
:103A3000F081E02D099508950F931F93CF93DF93A5
:103A4000EC016DE00E94141D8C016AE0CE010E9421
:103A5000141D800F911FDF91CF911F910F91089539
:103A60000F931F93CF93DF93EC010E94FA1C8C01FC
:103A7000CE010E941C1D800F911FDF91CF911F91DD
:103A80000F9108950F931F93CF93DF93EC010E9442
:103A9000141D8C01CE010E941C1D800F911FDF910F
:103AA000CF911F910F910895A1E2B0E0EAE5FDE109
:103AB0000C942D217C01C42EE52FCB01D22E19A20E
:103AC00021E02D1510F02AE0D22E8E010F5D1F4F40
:103AD0008D2C912CA12CB12C6C2D7E2FA501940145
:103AE0000E94E6208C2DD29E8019112401501109CC
:103AF0008A3010F4805D01C0895CF8018083211553
:103B000031054105510521F0C22EE32FCA01E4CF52
:103B1000B801C7010E94FA1CA196ECE00C9449215F
:103B2000A0E0B0E0E6E9FDE10C943121EC016A018E
:103B30007B012115310541F4E881F9810190F08183
:103B4000E02D642F09951DC02A303105A9F477FFB7
:103B500012C06DE20E94141D8C0144275527BA0142
:103B60004C195D096E097F092AE0CE010E94541D9F
:103B7000800F911F06C02AE0B701A601CE010E9466
:103B8000541DCDB7DEB7E8E00C944D210F931F9381
:103B9000CF93DF93EC019A01AB01662757FD609547
:103BA000762F0E94901D8C01CE010E941C1D800F5B
:103BB000911FDF91CF911F910F910895211531052C
:103BC00049F4DC01ED91FC910190F081E02D642F2E
:103BD000099508950E94541D08959A01462F50E0BA
:103BE00060E070E00E94DE1D08959A01AB0160E084
:103BF00070E00E94DE1D0895FC0124853585F901E1
:103C0000E05CFF4F80819181F901EE5BFF4F2081E5
:103C10003181821B930B8F7399270895FC01848552
:103C20009585FC01E05CFF4F40815181FC01EE5B1A
:103C3000FF4F208131814217530741F00190F081FD
:103C4000E02DE80FF91F808190E008958FEF9FEF3E
:103C50000895FC0184859585FC01E05CFF4F40815F
:103C60005181FC01EE5BFF4F2081318142175307E8
:103C700079F0A081B181A80FB91F8C912081318189
:103C80002F5F3F4F2F7333273183208390E00895B8
:103C90008FEF9FEF0895FC0181A1882329F0A4896B
:103CA000B5898C9186FFFBCF11A20895CF93DF9346
:103CB000FC0126853785D901A05CBF4F8D919C9171
:103CC000119701968F739927E901CE5BDF4F4881E9
:103CD000598184179507D9F30D90BC91A02DA20F9F
:103CE000B31F6C93A685B785A05CBF4F11969C93BC
:103CF0008E93A689B7892C9181E090E0078C02C051
:103D0000880F991F0A94E2F7282B2C9381E081A356
:103D10000488F589E02D80818064808381E090E0D3
:103D2000DF91CF91089508951F920F920FB60F92D1
:103D300011242F933F934F938F939F93EF93FF9370
:103D40008091C00082FD1CC04091C6008091B004EB
:103D50009091B10401968F7399272091B20430910C
:103D6000B3048217930771F0E091B004F091B104AD
:103D7000E059FB4F40839093B1048093B00402C09C
:103D80008091C600FF91EF919F918F914F913F914C
:103D90002F910F900FBE0F901F9018958AE094E01E
:103DA0000E94FC1D892B11F00E94931E08951F9202
:103DB0000F920FB60F9211242F933F938F939F93DF
:103DC000EF93FF9320916C0430916D0480916E0409
:103DD00090916F042817390731F48091C1008F7DCD
:103DE0008093C10014C0E0916E04F0916F04E45D13
:103DF000FB4F208180916E0490916F0401968F7328
:103E0000992790936F0480936E042093C600FF91CE
:103E1000EF919F918F913F912F910F900FBE0F9037
:103E20001F901895A0E0B0E0E8E1FFE10C942D218F
:103E3000FC011382128288EE93E0A0E0B0E084835C
:103E40009583A683B7838EEB92E0918380837587F9
:103E5000648757874687318B208B138B028BF58ABB
:103E6000E48AD78AC68AB18EA08E938E828E8F8581
:103E7000848F8889858F8989868F8A89878F8B89A6
:103E800080A3ECE00C944921CF92DF92EF92FF9255
:103E9000CF93DF93EC016A017B01411581EE580756
:103EA00061057105F9F0EC89FD8981E090E008A0D9
:103EB00002C0880F991F0A94E2F7808360E079E0DE
:103EC0008DE390E0A70196010E94E6202150310980
:103ED000410951095695479537952795211580E158
:103EE000380798F0EC89FD89108260E874E88EE16B
:103EF00090E0A70196010E94E62021503109410976
:103F000051095695479537952795E889F989308362
:103F1000EA89FB89208319A2EE89FF89408181E02B
:103F200090E09C010C8C02C0220F331F0A94E2F730
:103F3000422B4083EE89FF8940819C010D8C02C099
:103F4000220F331F0A94E2F7422B4083EE89FF8948
:103F500040819C010E8C02C0220F331F0A94E2F7AD
:103F6000422B4083EE89FF8920810F8C02C0880F8D
:103F7000991F0A94E2F7809582238083DF91CF9185
:103F8000FF90EF90DF90CF900895BF92CF92DF9295
:103F9000EF92FF92CF93DF93EC016A017B01B22E87
:103FA000411581EE580761057105F9F0EC89FD892D
:103FB00081E090E008A002C0880F991F0A94E2F700
:103FC000808360E079E08DE390E0A70196010E9494
:103FD000E6202150310941095109569547953795F9
:103FE0002795211580E1380798F0EC89FD8910822A
:103FF00060E874E88EE190E0A70196010E94E62057
:104000002150310941095109569547953795279512
:10401000E889F9893083EA89FB892083E88DF98D65
:10402000B082EE89FF89408181E090E09C010C8C98
:1040300002C0220F331F0A94E2F7422B4083EE891D
:10404000FF8940819C010D8C02C0220F331F0A940E
:10405000E2F7422B4083EE89FF8940819C010E8C60
:1040600002C0220F331F0A94E2F7422B4083EE89ED
:10407000FF8920810F8C02C0880F991F0A94E2F7F4
:10408000809582238083DF91CF91FF90EF90DF9026
:10409000CF90BF9008958F929F92AF92BF92CF9290
:1040A000DF92EF92FF920F931F9381E08F9385E051
:1040B0008F9387E08F9383E08F9384E08F93E6EC78
:1040C0008E2E912CF2ECAF2EB12CA1ECCA2ED12C5D
:1040D000B0ECEB2EF12C04EC10E025EC30E04CE2DF
:1040E00054E060E774E08AE094E00E94121F0F90B1
:1040F0000F900F900F900F901F910F91FF90EF90E6
:10410000DF90CF90BF90AF909F908F9008950E94C6
:10411000C21B0E945A12CEECDEE10E944C16209780
:10412000E1F30E94CE1EF9CFA29FB001B39FC00160
:10413000A39F700D811D1124911DB29F700D811DD3
:104140001124911D08950E949420A59F900DB49F65
:10415000900DA49F800D911D11240895B7FF0C941C
:10416000A3200E94A320821B930B0895DB018F9351
:104170009F930E94A320BF91AF91A29F800D911D9C
:10418000A39F900DB29F900D11240895991B79E083
:1041900004C0991F961708F0961B881F7A95C9F7D7
:1041A00080950895AA1BBB1B51E107C0AA1FBB1F26
:1041B000A617B70710F0A61BB70B881F991F5A95B3
:1041C000A9F780959095BC01CD010895A1E21A2E22
:1041D000AA1BBB1BFD010DC0AA1FBB1FEE1FFF1FAB
:1041E000A217B307E407F50720F0A21BB30BE40BFB
:1041F000F50B661F771F881F991F1A9469F7609542
:104200007095809590959B01AC01BD01CF010895FB
:10421000052E97FB1EF400940E941F2157FD07D026
:104220000E94E62007FC03D04EF40C941F21509509
:104230004095309521953F4F4F4F5F4F0895909592
:104240008095709561957F4F8F4F9F4F08952F9266
:104250003F924F925F926F927F928F929F92AF9216
:10426000BF92CF92DF92EF92FF920F931F93CF9363
:10427000DF93CDB7DEB7CA1BDB0B0FB6F894DEBFFA
:104280000FBECDBF09942A88398848885F846E8420
:104290007D848C849B84AA84B984C884DF80EE806A
:1042A000FD800C811B81AA81B981CE0FD11D0FB673
:1042B000F894DEBF0FBECDBFED010895EE0FFF1FD6
:1042C0000590F491E02D0994FB01DC0102C00190FE
:1042D0000D9241505040D8F70895F999FECF92BD04
:1042E00081BDF89A992780B50895262FF999FECFB8
:1042F0001FBA92BD81BD20BD0FB6F894FA9AF99A03
:0A4300000FBE01960895F894FFCF58
:10430A000000B404200008409CFF0088130002004B
:10431A000200020002000200020002000200020083
:10432A000200020002000200020002000200200154
:10433A00270121022B03220326042304260524062F
:10434A002506280629062A8025000005400AA120FC
:10435A004EA50020244EA52C2330C01200001A407E
:10436A000AA1204EA5001B1E27522C2330802500AF
:10437A000005400AA1204EA50020244EA52C23307A
:10438A00004B000006400AD0009D49007B289D4949
:10439A002C233000E1000005400A4501D7DC03B8B0
:1043AA001E0EBF00232E48E801008A400A6001550C
:1043BA005502AD1E20000023C80154582074696DAF
:1043CA00656F7574210057616974696E6720626947
:1043DA006E640A00476F7420706B740A006461741B
:1043EA006120676F6F640A007363616E6E65722085
:1043FA006D6F6465004F70656E4C52536E67205244
:10440A0058207374617274696E672000206F6E2081
:10441A004857200053617665642062696E6420649F
:10442A0061746120746F20454550524F4D0A00490E
:10443A0020616D20736C61766500456E74657269E2
:10444A006E67206E6F726D616C206D6F64650045DA
:10445A004550524F4D2064617461206E6F7420760E
:10446A00616C6964206F722062696E64206A756D7E
:10447A0070706572207365742C20666F7263696E42
:10448A00672062696E640A0052582068616E67008C
:10449A00B200F4014C0300070B0C101115000A03BB
:1044AA000E121300010400000000080001000010B1
:1044BA000000200000000100000200000000561E5B
:0A44CA00D81CFC1D291E0E1E4B1EFF
:107E00000F92CDB7DEB7112484B714BE81FFF1D035
:107E100082E08093C00088E18093C10086E0809377
:107E2000C20080E18093C4008EE0CDD088249924E4
:107E3000CC24C394F5E0DF2EE1E1EE2E73E0F72EC3
:107E4000B6D0082F813479F4B2D08983C2D0898129
:107E5000823811F481E005C0813811F485E001C059
:107E600083E09ED09AC0823411F484E103C085344B
:107E700019F485E0B6D091C0853561F498D0082F0B
:107E800010E095D090E0982E8824802A912A880CC2
:107E9000991C82C0863521F484E0A3D080E0E1CF34
:107EA000843609F04CC083D082D0A82E80D0B82E62
:107EB00000E011E07CD0F80181938F01AE16D1F77C
:107EC00088D0FB2DF53489F4E0E0F1E00BC0F9999E
:107ED000FECF92BC81BC0894811C911C819180BD15
:107EE000FA9AF99AEA1598F358C08B2D863409F05E
:107EF00054C0F401F7BEE89507B600FCFDCFF401CD
:107F0000A0E0B1E02C9130E011968C91119790E0B7
:107F1000982F8827822B932B12960C01C7BEE895C9
:107F20001124329681E0A038B80761F7F401D7BE7A
:107F3000E89507B600FCFDCFE7BEE8952EC0843774
:107F4000F1F435D034D0182F32D0B82E42D0FB2DDA
:107F5000F63421F4F40105914F010CC0FB2DF534EA
:107F600049F4F999FECF92BC81BC0894811C911C04
:107F7000F89A00B5802F14D0115049F70EC08537FC
:107F800039F427D08EE10CD085E90AD08FE069CF93
:107F9000813511F488E017D01CD080E101D050CF9A
:107FA0009091C00095FFFCCF8093C600089580910A
:107FB000C00087FFFCCF8091C00084FD01C0A89560
:107FC0008091C6000895E0E6F0E098E19083808318
:107FD0000895EDDF803219F088E0F5DFFFCF84E10E
:107FE000DFCF1F93182FE3DF1150E9F7F2DF1F9166
:0E7FF0000895282E80E0E7DFEE27FF27099492
:027FFE0001057B
:0400000300007E007B
:00000001FF
